:020000040000FA
:10000000F26A72EF01F0FFFFB6EF10F0FFFFFFFFA3
:10001000FFFFFFFFFFFFFFFFB8EF10F0A96EA69EE6
:10002000A69CA680A8501200A86EA69EA69CA68498
:10003000F29EF2BE18EF00F0550EA76EAA0EA76E44
:10004000A682F28EA6941200C70ED56E940ED66EBE
:10005000F294F2A429EF00F0120024EC00F024EC5A
:1000600000F024EC00F024EC00F024EC00F024EC90
:1000700000F024EC00F024EC00F024EC00F024EC80
:1000800000F012002DEC00F02DEC00F02DEC00F053
:100090002DEC00F02DEC00F02DEC00F02DEC00F03C
:1000A0002DEC00F02DEC00F02DEC00F0120052ECE5
:1000B00000F037EC00F012000A0EA96EFF0E14ECEF
:1000C00000F024EC00F012000A0EA96E5A0E14EC97
:1000D00000F024EC00F01200A68EF86A000EF76E15
:1000E000000EF66EFE0E606F3F0E616FED0E626FDA
:1000F000DE0E636F0900F550631B0900F550621BAB
:10010000020E605F000E615B60516111D8A47AEF4E
:1001100000F0621F631F0900F550635DD8A4A2EFD1
:1001200000F00900F550625DD8A4A2EF00F00A0EBD
:100130000EEC00F05A0AD8B4D5EF01F064EC00F0F0
:1001400097EF00F08B928B9042EC00F00A0E606FFC
:100150008B8057EC00F08B9057EC00F0602FA8EFED
:1001600000F0A2EF00F0A68EF86A3F0EF76EFC0ECC
:10017000F66E000E606F400E616FED0E626FDE0E68
:10018000636F0900F550631B0900F550621B020EF6
:10019000605F000E615B60516111D8A4C1EF00F097
:1001A000621F631F62516311D8A46CEF00F0A68E2A
:1001B000F86A3F0EF76EFA0EF66E0900F550676F9B
:1001C0000900F550666FA68EF86A7F0EF76EF60E80
:1001D000F66E0900F550696F0900F550686F6651B9
:1001E000685D67516959D8A06CEF00F08B828B80F5
:1001F000F00E606F000E616FF86A040EF76E000E6D
:10020000F66EA68EA69CA688A684550EA76EAA0E8C
:10021000A76EA682400EF626D8B0F72A010E605FC0
:10022000000E615B60516011D8A401EF01F0000E77
:10023000606F3C0E616FF86A040EF76E000EF66E8A
:100240000900FF0EF55CD8A4F6EF00F0010E605F28
:10025000000E615B60516111D8A420EF01F0F00E37
:10026000616FF86A040E656F000E646F61A98B9070
:1002700061B98B8064C0F6FF65C0F7FF000EF626FB
:10028000400EF72200EE6BF0400E606F0900F5CFD4
:10029000EEFF602F46EF01F064C0F6FF65C0F7FF88
:1002A00000EE6BF0400E606FEECFF5FF0D00602F9B
:1002B00054EF01F064C0F6FF65C0F7FFA68EA69C60
:1002C000A698A684550EA76EAA0EA76EA682400E0B
:1002D0006427D8B0652B612F36EF01F08B928B909D
:1002E00064EC00F0000E806E400E816E400E826E57
:1002F0003E0E926E820E936EA00E946E2C0EE8CF80
:1003000038FF000EE8CF39FF200EE8CF3AFF000E8D
:10031000E8CFC1FF3E0EE8CFC0FF000EE8CF79FF67
:10032000E8CF78FFE8CF77FFF19E000179EF03F087
:100330000A0E0EEC00F05A0AD8A4B3EF00F0A68E15
:10034000F86A000EF76E000EF66EFE0E606F3F0E3E
:10035000616FED0E626FDE0E636F0900F550631B77
:100360000900F550621B020E605F000E615B605178
:100370006111D8A4ADEF01F0621F631F0900F550B1
:10038000635DD8A4B3EF00F00900F550625DD8A416
:10039000B3EF00F00A0E0EEC00F05A0AD8B4D5EF15
:1003A00001F064EC00F0CAEF01F079EF03F0FFFF19
:1003B000FFFFFFFFFFFFFFFFFFFFFFFFFFFFFFFF4D
:1003C000FFFFFFFFFFFFFFFFFFFFFFFFFFFFFFFF3D
:1003D000FFFFFFFFFFFFFFFFFFFFFFFFFFFFFFFF2D
:1003E000FFFFFFFFFFFFFFFFFFFFFFFFFFFFFFFF1D
:1003F000FFFFFFFFFFFFFFFFFFFFFFFFFFFFFFFF0D
:100400004154000041544530000041542B434C54AA
:10041000533D3100000041542657000041542B4306
:10042000434C4B3F000041542B434D47463D310068
:10043000000041542B435245473F000041542B4399
:100440004D47533D220000002B32373832353130D2
:10045000353738322200000043656E7465722050D3
:1004600069766F74204F41313720000041542B438F
:100470004D474C3D22414C4C2200000041542B433F
:100480004D47533D000041542B434D47443D000030
:1004900041542B435351000041542B43494D4900D3
:1004A000000041542B43474154543F000000415445
:1004B0002B53415042523D332C312C22434F4E544A
:1004C000595045222C2247505253220000004154DB
:1004D0002B53415042523D332C312C2241504E225D
:1004E0002C22494E5445524E45542200000041549E
:1004F0002B53415042523D312C31000041542B537B
:10050000415042523D322C31000041542B4854544A
:1005100050494E495400000041542B485454505007
:100520004152413D22434944222C310000004154B4
:100530002B48545450504152413D2255524C222C8C
:1005400022687474703A2F2F6661726D696E672E1F
:100550006167726967656C2E636F2E7A612F696EB1
:100560006465782F6170692F6170695F646174617F
:100570002E7068702200000041542B485454505093
:100580004152413D22434F4E54454E54222C22614C
:1005900070706C69636174696F6E2F782D777777EF
:1005A0002D666F726D2D75726C656E636F64656418
:1005B0002200000041542B48545450444154413DC2
:1005C00000002C313030303000006E616D653D61CF
:1005D0006A61785F70696E6700006E616D653D727B
:1005E0006426646174613D33413831000000304459
:1005F000000041542B48545450414354494F4E3D00
:100600003100000041542B4854545052454144009D
:10061000000041542B485454505445524D000000A2
:1006200041542B53415042523D302C3100004F4B2E
:100630000000415400004154453000004552524FE3
:10064000520000002B435245473A20302C31000025
:100650002B435245473A20302C35000041542B4360
:1006600050494E3F00002B4350494E3A20524541DD
:10067000445900002B4350494E3A2053494D2050D5
:10068000494E00002B435343413A00002B434D4752
:10069000533A00002B434D474C3A00002B4347414F
:1006A00054543A20310000002B53415042523A003A
:1006B0000000444F574E4C4F414400002B485454C7
:1006C00050414354494F4E3A00002B485454505225
:1006D0004541443A00002B485454505445524D0073
:1006E00000002B43434C4B3A00002B4353513A003C
:1006F00000004CEF05F00A0A0A0A0A0A0A0A0A0A66
:100700000D4167726967656C20466C6F7720436F97
:100710006E74726F6C2056616C76652000000A0A58
:100720000D3F203D20436F6D6D616E642048656C08
:10073000700A0A0D000061203D204175746F6D61E3
:100740007469630A0D00000063203D20436C6F73E1
:10075000652076616C7665203120737465702C207D
:10076000284F4E4C5920494E204D414E55414C2961
:100770000A0D000043203D20436C6F7365207661B5
:100780006C7665203130302073746570732C2028AE
:100790004F4E4C5920494E204D414E55414C290A4F
:1007A0000D00000064203D2044656372656D656E38
:1007B000742076616C7665206E756D6265720A0DC7
:1007C000000066203D20466C6F77206D6574657271
:1007D00020646174610A0D00000069203D20496EAB
:1007E0006372656D656E742076616C7665206E75DA
:1007F0006D6265720A0D00006B203D204B616C69D3
:1008000062726174696F6E0A0D0000006D203D20F8
:100810004D616E75616C0A0D00006F203D204F70B8
:10082000656E2076616C7665203120737465702C5E
:1008300020284F4E4C5920494E204D414255414CA5
:10084000290A0D0000004F203D204F70656E207674
:10085000616C7665203130302073746570732C20A4
:10086000284F4E4C5920494E204D414E55414C2960
:100870000A0D000070203D205061636B6574206498
:100880006174610A0D00000072203D20526573659D
:100890007420666C6F772070756C736520636F755C
:1008A0006E7465720A0D000076203D2056616C76EC
:1008B0006520646174610A0D0A0D0000356D7320B6
:1008C0002020454550202020434F4D0A0D000000B8
:1008D000356D7320202020505620202020202053CA
:1008E000502020202020204E455720202020205519
:1008F000464F320A0D000000436F756E740A0D00FA
:100900000000202020202020202020202020202027
:100910002020000043656E7465725069766F7446DE
:100920006C6F77200000436F6E74726F6C6C657231
:10093000204F4131372000004155544F4D4154491B
:1009400043202020202020200000202020202020C4
:100950002020202020202020202000004D414E5526
:10096000414C20202020202020202020000020207A
:1009700020202020202020202020202020200000B7
:10098000202020456469743F204E6F2020202020C5
:100990000000202020456469743F205965732020A1
:1009A0002020000053657474696E6773204D656E76
:1009B000753A2020000053657420706F696E743A98
:1009C00020000000466C6F772073657420706F699B
:1009D0006E743A200000466C6F7720726174652057
:1009E00069733A202020000053656C656374204DC4
:1009F0004F44453A20202020000020202020204D78
:100A0000414E55414C202020202000002020202055
:100A1000204155544F4D4154494320200000464148
:100A2000554C542072656C61793A202020200000DA
:100A30002020202020454E41424C452020202020CF
:100A40000000202020202044495341424C452020D2
:100A500020200000534D532070696E2E2E2E3A2018
:100A60000000534D532070696E3A20202020202032
:100A700020200000212120464C4F57204641554C54
:100A8000542021210000202020504F57455220445F
:100A90004F574E202020000001011F0EAF6E010EA7
:100AA000B06E080EB86E260EAC6E900EAB6E230EB6
:100AB000756E000E766E080E706E220E726E980EB7
:100AC000716ECF68CE68810ECD6E6C0EBB6EBC6A47
:100AD0003E0EBA6E330EB16E000EB46E4E6AB36A3D
:100AE000B26A010E6E6F6F6B706B020E716F726B7C
:100AF000736B030E746F756B766B040E776F786B88
:100B0000796B050E7A6F7B6B7C6B060E7D6F7E6B4F
:100B10007F6B070E806F816B826B080E836F846B17
:100B2000856B090E866F876B886B0A0E896F8A6BDF
:100B30008B6BF26A9F6AA26AA56AF08CF08E9F8026
:100B4000A282F19AF1989D8AA38A9D809D82A192AA
:100B5000A082F086F088006A016A026A036A046A69
:100B6000056A066A076A086A346B356B080E186EE8
:100B7000640E366FC80E376FAE6B028C0A0E4B6E6A
:100B80004C6A000E4D6E000E5F6FB16BB26BF90ECA
:100B9000386F396F3E0E3A6F3B6F7F0E3C6F3D6F83
:100BA000FF0E3E6F3F6FB2CF4CF1B3CF4DF14EC051
:100BB0004EF1A56BA66BA76BB2CF55F1B3CF56F133
:100BC0004EC057F1AA6BAB6BAC6B020E5D6F020EA1
:100BD0005E6F3C0E476E000E486ED00E496E070EDB
:100BE0004A6E100E996F270E9A6F000E9B6FA16FC1
:100BF000A26F000E516E000E536E000E506E000E6E
:100C0000526E000EBC6FFF0EB56F000E0EEC00F0C2
:100C1000996F010E0EEC00F09A6F020E0EEC00F0D0
:100C2000076E030E0EEC00F0EA6F040E0EEC00F0FF
:100C3000EB6F050E0EEC00F0EC6F060E0EEC00F004
:100C4000ED6F1DEC2FF0C80E9C5DD8A02AEF06F0CA
:100C5000640E9C6FE80E9D6F9F6F030E9E6FA06FDA
:100C6000D890A0339F33D890A0339F33676B828690
:100C7000949694880000000000000000000000002E
:100C8000000000000000000000000000080E186EC8
:100C9000000E196E4DEC18F01950E3EC18F0D3EC7F
:100CA00023F04CEC00F04DEC18F01950E3EC18F088
:100CB000300E196E43EC19F0F2EC0FF043EC19F022
:100CC000F2EC0FF043EC19F0F2EC0FF0200E196E7D
:100CD00043EC19F0F2EC0FF0280EF8EC1FF0F2ECF8
:100CE0000FF0080EF8EC1FF0F2EC0FF0010EF8EC2C
:100CF0001FF0F2EC0FF0F2EC0FF00C0EF8EC1FF01E
:100D0000F2EC0FF0800EF8EC1FF0F2EC0FF0090E91
:100D1000186E126B040E176F8A0E1E6F170E1F6F60
:100D200081A2179781B21787A86B81A4129381B40F
:100D30001283AD6BFF0EB66F420E126E8A8A276A5F
:100D4000286AC80EB86F000EB96F606B616BD08EE9
:100D5000F28EF28C020EE86F040EE96FA68EF86A2E
:100D6000060EF76EF60EF66E2AEC24F08AEC24F0EE
:100D7000A68EF86A070EF76E1E0EF66E2AEC24F0A9
:100D8000E9EC0DF05250D8B4AEEC0BF01FEC0FF0C4
:100D90009EEC24F0D1EC06F006807AEC28F0C0EF4F
:100DA00006F0FB6A0D0EFA6E5250E834E8347C0B04
:100DB000B80FD8B0FA2AF96E24EF07F02BEF07F03E
:100DC0004CEF07F06EEF07F08FEF07F0B8EF07F08A
:100DD000DAEF07F0FBEF07F024EF08F048EF08F038
:100DE0006CEF08F090EF08F0B5EF08F0E3EF08F0D3
:100DF000F8EF08F0FBEF08F029EF09F03EEF09F0FB
:100E000041EF09F06EEF09F090EF09F0B1EF09F052
:100E1000E3EF09F006EF0AF029EF0AF04CEF0AF0D1
:100E20006BEF0AF020EF07F020EF07F020EF07F05C
:100E300020EF07F020EF07F020EF07F020EF07F09A
:100E4000000E526ED2EF0AF004AA29EF07F0049ABE
:100E5000522AD2EF0AF0A68EF86A090EF76EA40E97
:100E6000F66E38EC24F0A68EF86A090EF76E920E34
:100E7000F66E47EC24F0C90EF8EC1FF0F2EC0FF020
:100E80000F0EF8EC1FF0F2EC0FF0049204980490AF
:100E9000049A522AD2EF0AF004A254EF07F0049207
:100EA000522A522A6CEF07F004B85AEF07F004A058
:100EB0006CEF07F004980490A68EF86A090EF76E9E
:100EC000800EF66E47EC24F0C90EF8EC1FF0F2EC41
:100ED0000FF0522AD8EF07F0D2EF0AF004A275EF14
:100EE00007F00492526A8DEF07F004B87BEF07F029
:100EF00004A08DEF07F004980490A68EF86A090EFE
:100F0000F76E920EF66E47EC24F0C90EF8EC1FF067
:100F1000F2EC0FF05206D8EF07F0D2EF0AF0A68EEF
:100F2000F86A090EF76EB60EF66E38EC24F08B0EEA
:100F3000B76F99512B6E9A512C6E56EC24F0A68EF9
:100F4000F86A090EF76E800EF66E47EC24F0C90EB3
:100F5000F8EC1FF0F2EC0FF00F0EF8EC1FF0F2ECD3
:100F60000FF0049204980490049A522AD2EF0AF0E7
:100F700004A2C0EF07F00492070E5226D8EF07F044
:100F800004B8C6EF07F004A0D8EF07F00498049067
:100F9000A68EF86A090EF76E920EF66E47EC24F0F4
:100FA000C90EF8EC1FF0F2EC0FF0522AD8EF07F060
:100FB000D2EF0AF004A2E1EF07F00492522AF9EF0F
:100FC00007F004B8E7EF07F004A0F9EF07F0049882
:100FD0000490A68EF86A090EF76E800EF66E47EC46
:100FE00024F0C90EF8EC1FF0F2EC0FF05206F9EF06
:100FF00007F0D2EF0AF0A68EF86A090EF76EC40E5B
:10100000F66E38EC24F0A68EF86A090EF76E020E22
:10101000F66E47EC24F0C60EB76F99512B6E9A51BD
:101020002C6E72EC24F0C90EF8EC1FF0F2EC0FF00D
:101030000F0EF8EC1FF0F2EC0FF0049204980490FD
:10104000049A522AD2EF0AF004A83CEF08F0049860
:101050002E2A0A0E2E5C000ED8B02E6EC90EF8ECA9
:101060001FF0F2EC0FF02E50300FFFEC1FF0C90E06
:10107000F8EC1FF0F2EC0FF004A246EF08F0049237
:10108000C80EF8EC1FF0F2EC0FF0522AD2EF0AF083
:1010900004A860EF08F004982F2A0A0E2F5C000EB7
:1010A000D8B02F6EC80EF8EC1FF0F2EC0FF02F50F6
:1010B000300FFFEC1FF0C80EF8EC1FF0F2EC0FF051
:1010C00004A26AEF08F00492C70EF8EC1FF0F2ECED
:1010D0000FF0522AD2EF0AF004A884EF08F0049827
:1010E000302A0A0E305C000ED8B0306EC70EF8EC15
:1010F0001FF0F2EC0FF03050300FFFEC1FF0C70E76
:10110000F8EC1FF0F2EC0FF004A28EEF08F004925E
:10111000C60EF8EC1FF0F2EC0FF0522AD2EF0AF0F4
:1011200004A8A8EF08F00498312A0A0E315C000EDA
:10113000D8B0316EC60EF8EC1FF0F2EC0FF0315063
:10114000300FFFEC1FF0C60EF8EC1FF0F2EC0FF0C2
:1011500004A2B3EF08F0049230EC14F02B50996F16
:101160002C509A6F522AD2EF0AF0A68EF86A090E16
:10117000F76EE80EF66E38EC24F007A0CAEF08F020
:10118000A68EF86A090EF76EFA0EF66E47EC24F09A
:10119000D2EF08F0A68EF86A0A0EF76E0C0EF66E05
:1011A00047EC24F0C50EF8EC1FF0F2EC0FF00F0E38
:1011B000F8EC1FF0F2EC0FF0049204980490049AFB
:1011C000522AD2EF0AF004B8E9EF08F004A0EFEFDA
:1011D00008F00498049007705206F6EF08F004A295
:1011E000F6EF08F00492522AF6EF08F0D2EF0AF078
:1011F000522AD2EF0AF0A68EF86A0A0EF76E1E0E79
:10120000F66E38EC24F007A210EF09F0A68EF86A0B
:101210000A0EF76E300EF66E47EC24F018EF09F068
:10122000A68EF86A0A0EF76E420EF66E47EC24F0B0
:10123000C50EF8EC1FF0F2EC0FF00F0EF8EC1FF0FB
:10124000F2EC0FF0049204980490049A522AD2EF20
:101250000AF004B82FEF09F004A035EF09F0049864
:101260000490077252063CEF09F004A23CEF09F02B
:101270000492522A3CEF09F0D2EF0AF0522AD2EF40
:101280000AF0A68EF86A0A0EF76E540EF66E38EC67
:1012900024F0EA51FFEC1FF0EB51FFEC1FF0EC5192
:1012A000FFEC1FF0ED51FFEC1FF0A68EF86A090E5F
:1012B000F76E800EF66E47EC24F0C90EF8EC1FF0C6
:1012C000F2EC0FF00F0EF8EC1FF0F2EC0FF00492BE
:1012D00004980490049A522AD2EF0AF004A276EFFE
:1012E00009F00492070E52268EEF09F004B87CEF45
:1012F00009F004A08EEF09F004980490A68EF86A15
:10130000090EF76E920EF66E47EC24F0C90EF8EC5B
:101310001FF0F2EC0FF0522A8EEF09F0D2EF0AF034
:1013200004A297EF09F00492522AAFEF09F004B833
:101330009DEF09F004A0AFEF09F004980490A68E89
:10134000F86A090EF76E800EF66E47EC24F0C90EAF
:10135000F8EC1FF0F2EC0FF05206AFEF09F0D2EF0D
:101360000AF0A68EF86A0A0EF76E620EF66E38EC78
:1013700024F0A68EF86A090EF76E020EF66E47ECA0
:1013800024F0C60EF8EC1FF0F2EC0FF0EA51FFEC7F
:101390001FF0EB51FFEC1FF0EC51FFEC1FF0ED5193
:1013A000FFEC1FF0C90EF8EC1FF0F2EC0FF00F0E7F
:1013B000F8EC1FF0F2EC0FF0049204980490049AF9
:1013C000522AD2EF0AF004A8FAEF09F00498ED2BA4
:1013D0003A0EED5D300ED8B0ED6FC90EF8EC1FF08F
:1013E000F2EC0FF0ED51FFEC1FF0C90EF8EC1FF01E
:1013F000F2EC0FF004A204EF0AF00492C80EF8EC2D
:101400001FF0F2EC0FF0522AD2EF0AF004A81DEF01
:101410000AF00498EC2B3A0EEC5D300ED8B0EC6F6D
:10142000C80EF8EC1FF0F2EC0FF0EC51FFEC1FF0DF
:10143000C80EF8EC1FF0F2EC0FF004A227EF0AF050
:101440000492C70EF8EC1FF0F2EC0FF0522AD2EF24
:101450000AF004A840EF0AF00498EB2B3A0EEB5D7B
:10146000300ED8B0EB6FC70EF8EC1FF0F2EC0FF0B7
:10147000EB51FFEC1FF0C70EF8EC1FF0F2EC0FF091
:1014800004A24AEF0AF00492C60EF8EC1FF0F2EC48
:101490000FF0522AD2EF0AF004A863EF0AF0049882
:1014A000EA2B3A0EEA5D300ED8B0EA6FC60EF8ECC1
:1014B0001FF0F2EC0FF0EA51FFEC1FF0C60EF8EC53
:1014C0001FF0F2EC0FF004A269EF0AF00492070E8D
:1014D000525ED2EF0AF0000E0EEC00F0995DD8B427
:1014E00079EF0AF0995114EC00F0E9EC0FF06BEF92
:1014F0000AF0010E0EEC00F09A5DD8B487EF0AF006
:101500009A5114EC00F0E9EC0FF079EF0AF0020EBA
:101510000EEC00F0075CD8B495EF0AF0075014EC1D
:1015200000F0E9EC0FF087EF0AF0030E0EEC00F08C
:10153000EA5DD8B4A3EF0AF0EA5114EC00F0E9EC4C
:101540000FF095EF0AF0040E0EEC00F0EB5DD8B44E
:10155000B1EF0AF0EB5114EC00F0E9EC0FF0A3EF5F
:101560000AF0050E0EEC00F0EC5DD8B4BFEF0AF007
:10157000EC5114EC00F0E9EC0FF0B1EF0AF0060EBC
:101580000EEC00F0ED5DD8B4CDEF0AF0ED5114ECA7
:1015900000F0E9EC0FF0BFEF0AF0040E506E526A53
:1015A000D2EF0AF012001200000E386E000E396EF3
:1015B000280E3A6E010E3B6E000E3C6EA5C13DF04A
:1015C000A6C13EF0A7C13FF0406A416A76EC15F033
:1015D000090E8C6F01EE6EF0EE2EFCEF0AF0ED506E
:1015E000E9CF90F1EACF91F1090EEE6E38C0EEFF2F
:1015F00039C0EEFFFEEF0AF0EE50EE508C2FECEF0C
:101600000AF090C1E9FF91C1EAFF6E0EE95CD8A42F
:101610000FEF0BF0010EEA58D8B431EF0BF0860E45
:10162000E95CD8A419EF0BF0010EEA58D8B468EFC2
:101630000BF0EE50EE50EE50EE503850EE5C39505C
:10164000EE58D8A031EF0BF0080EE95E000EEA5A12
:10165000EE50385CEE503958D8A068EF0BF09DEF93
:101660000BF090C1E9FF91C1EAFF90C1E1FF91C188
:10167000E2FF860EE95CD8A443EF0BF0010EEA58B6
:10168000D8B466EF0BF0EE50EE50EE50EE503850FE
:10169000EE5C3950EF58D8B066EF0BF0EDCF8FF11C
:1016A000EDCF8EF1EFCF8DF1E6CFEEFFE6CFEEFF7F
:1016B000E7CFEFFF8FC1E5FF8EC1E5FF8DC1E6FFEC
:1016C000E650E650ED50ED5039EF0BF09DEF0BF08A
:1016D00090C1E9FF91C1EAFF90C1E1FF91C1E2FF32
:1016E0006E0EE95CD8A47AEF0BF0010EEA58D8B47C
:1016F0009BEF0BF0ED50ED50EE50385CEF50395849
:10170000D8B09BEF0BF0EDCF8FF1EDCF8EF1EFCF97
:101710008DF1E6CFEEFFE6CFEEFFE7CFEFFF8FC113
:10172000E5FF8EC1E5FF8DC1E5FFE550E550ED50C9
:10173000ED5070EF0BF09DEF0BF07BC138F07CC1EA
:1017400039F03A6A3B6A3C6A38C0A1F139C0A2F16B
:10175000A151F227A251F323F42B1200FB6A170EBA
:10176000FA6E5050E834E8347C0B720FD8B0FA2A85
:10177000F96EFDEF0BF001EF0CF019EF0CF022EF1A
:101780000CF036EF0CF04AEF0CF057EF0DF05BEF7A
:101790000DF06FEF0DF0C2EF0DF0C6EF0DF0F9EFA9
:1017A0000BF0F9EF0BF0F9EF0BF0F9EF0BF0F9EFAD
:1017B0000BF0F9EF0BF0F9EF0BF0F9EF0BF0F9EF9D
:1017C0000BF0F9EF0BF0F9EF0BF0F9EF0BF0F9EF8D
:1017D0000BF0F9EF0BF0F9EF0BF0F9EF0BF0F9EF7D
:1017E0000BF0F9EF0BF0F9EF0BF0F9EF0BF0F9EF6D
:1017F0000BF0000E506EAEEF0BF0010E506ED9EFF5
:101800000DF0A68EF86A090EF76E140EF66E38EC1F
:1018100024F0A68EF86A090EF76E260EF66E47ECD7
:1018200024F0FA0E106E000E116E020E506ED9EFFB
:101830000DF010501110D8A420EF0CF0030E506ED4
:10184000D9EF0DF0A68EF86A090EF76E020EF66E4D
:1018500038EC24F0A68EF86A090EF76E020EF66ECA
:1018600047EC24F0040E506ED9EF0DF0A68EF86A06
:10187000090EF76E380EF66E38EC24F0A68EF86A74
:10188000090EF76E4A0EF66E47EC24F0050E506E08
:1018900028EF00F007B052EF0CF060516111D8B49E
:1018A00056EF0CF0060E506E55EF0DF005AA55EFF1
:1018B0000DF0059A8A74C20EB76FF451D8A467EF81
:1018C0000CF0A1512B6EA2512C6E7EEF0CF0F2C1E8
:1018D00038F0F3C139F03A6A3B6A3C6AF4C13DF032
:1018E0003E6A3F6A406A416A76EC15F038C02BF0D8
:1018F00039C02CF038C0F5F139C0F6F1F26BF36B5A
:10190000F46B7EEC26F056EC24F0DAEC0DF0FFECF4
:101910001FF0C80EB76F99512B6E9A512C6E56EC72
:1019200024F055EF0DF09BB152EF0CF08A88B80E01
:10193000276E0B0E286E506E55EF0DF0F29E47503D
:101940004810F28ED8B497EC0FF003AC55EF0DF0C1
:10195000039CF29E9951A15D5A6F9A51A2595B6FF7
:10196000F28ED8A0B6EF0CF0BBEF0CF08AB8986BF3
:101970008A98C0EF0CF08AA8986B8A88C0EF0CF0A8
:101980005A515B11D8B454EF0DF0D8B0CEEF0CF033
:101990005A1F5B1F010E5A27000E5B23F40E5A5D7F
:1019A000010E5B59D8A0DDEF0CF0982B190E985D55
:1019B000190ED8B0986FDEEF0CF0986B880E5A5D58
:1019C000130E5B59D8A0EBEF0CF0800E5A6F000E8F
:1019D0005B6F3FEF0DF0600E5A5D090E5B59D8A0AA
:1019E000F8EF0CF0400E5A6F000E5B6F3FEF0DF0FA
:1019F000400E5A5D060E5B59D8A005EF0DF0200E83
:101A00005A6F000E5B6F3FEF0DF0900E5A5D010EA6
:101A10005B59D8A012EF0DF0100E5A6F000E5B6FDD
:101A20003FEF0DF0C80E5A5D000E5B59D8A01FEFB6
:101A30000DF0080E5A6F000E5B6F3FEF0DF0640E55
:101A40005A5D000E5B59D8A02CEF0DF0040E5A6FB2
:101A5000000E5B6F3FEF0DF00A0E5A5D000E5B59F2
:101A6000D8A039EF0DF0020E5A6F000E5B6F3FEFFA
:101A70000DF0000E5A6F000E5B6F3FEF0DF05A51E4
:101A8000275C5B512858D8B055EF0DF05AC127F0AC
:101A90005BC128F027502810D8B4272A9851272650
:101AA000000E282255EF0DF0986BD9EF0DF0070EC0
:101AB000506ED9EF0DF0A68EF86A090EF76E5C0E27
:101AC000F66E38EC24F0A68EF86A090EF76E6E0EEC
:101AD000F66E47EC24F0080E506E28EF00F007B0C9
:101AE0007BEF0DF060516111D8A47BEF0DF0090E72
:101AF000506EC0EF0DF005AAC0EF0DF0059A07B0CB
:101B00008AEF0DF08B0EB76F60512B6E61512C6E0A
:101B100056EC24F0C20EB76FF451D8A496EF0DF036
:101B2000A1512B6EA2512C6EADEF0DF0F2C138F029
:101B3000F3C139F03A6A3B6A3C6AF4C13DF03E6A4F
:101B40003F6A406A416A76EC15F038C02BF039C024
:101B50002CF038C0F5F139C0F6F1F26BF36BF46B91
:101B600056EC24F0DAEC0DF0FFEC1FF0C80EB76F66
:101B700099512B6E9A512C6E56EC24F0C0EF0DF05B
:101B8000D9EF0DF0040E506ED9EF0DF0A68EF86A65
:101B90000A0EF76E740EF66E38EC24F0A68EF86A14
:101BA0000A0EF76E860EF66E47EC24F08180D9EFB0
:101BB0000DF01200FB6A1B0EFA6E5350532AE834E4
:101BC000060BCA0FD8B0FA2AF96E2F0C2D0CCD0CCB
:101BD0007C0C190E04A2AF6F04A204EF0EF0190ED4
:101BE000B06FAE51D8A404EF0EF00F0EAE6F900E92
:101BF000606F010E616F8A98140EAF27FF0ED8B088
:101C0000AF6FAF51276E286A190E04A0B06F04A001
:101C10001FEF0EF0190EAF6FAE51D8A41FEF0EF0EC
:101C20000F0EAE6F900E606F010E616F8A88140EFA
:101C3000B027FF0ED8B0B06FB051276E286A1200DF
:101C4000C8EC26F0D8A01DEF0FF08B703F0AD8B477
:101C500064EF0EF05E0AD8B4EDEF0EF0200AD8B4AF
:101C6000EDEF0EF0220AD8B4F1EF0EF0200AD8B44E
:101C7000F7EF0EF0250AD8B4FDEF0EF0200AD8B425
:101C8000FDEF0EF02D0AD8B403EF0FF0200AD8B400
:101C900003EF0FF0260AD8B407EF0FF0200AD8B4EC
:101CA00007EF0FF0220AD8B40BEF0FF0200AD8B4D8
:101CB00011EF0FF0390AD8B417EF0FF0200AD8B49B
:101CC00017EF0FF01DEF0FF0A68EF86A060EF76EF5
:101CD000F60EF66E2AEC24F08AEC24F0A68EF86A52
:101CE000070EF76E1E0EF66E2AEC24F0A68EF86A2A
:101CF000070EF76E360EF66E2AEC24F0A68EF86A02
:101D0000070EF76E480EF66E2AEC24F0A68EF86ADF
:101D1000070EF76E740EF66E2AEC24F0A68EF86AA3
:101D2000070EF76EA40EF66E2AEC24F0A68EF86A63
:101D3000070EF76EC20EF66E2AEC24F0A68EF86A35
:101D4000070EF76EDA0EF66E2AEC24F0A68EF86A0D
:101D5000070EF76EF80EF66E2AEC24F0A68EF86ADF
:101D6000080EF76E0C0EF66E2AEC24F0A68EF86ABA
:101D7000080EF76E1A0EF66E2AEC24F0A68EF86A9C
:101D8000080EF76E460EF66E2AEC24F0A68EF86A60
:101D9000080EF76E740EF66E2AEC24F0A68EF86A22
:101DA000080EF76E880EF66E2AEC24F0A68EF86AFE
:101DB000070EF76EA40EF66E2AEC24F0A68EF86AD3
:101DC000080EF76EA80EF66E2AEC24F0C80E4B6EC5
:101DD000050E4C6E029C1DEF0FF0050E506E1DEFB0
:101DE0000FF08A88010E276E286A1DEF0FF08A888F
:101DF000640E276E286A1DEF0FF0019A019C000EF9
:101E00005F6F1DEF0FF0030E5F6F1DEF0FF0080EF9
:101E1000506E1DEF0FF08A98010E276E286A1DEF95
:101E20000FF08A98640E276E286A1DEF0FF0019A52
:101E3000019C020E5F6F1DEF0FF0120012005F5148
:101E4000020AD8A45EEF0FF0280E275C000E285877
:101E5000D8A02EEF0FF0280E2FEF0FF02750096EAD
:101E60008AA85EEF0FF0280E0A6E09500A5C0B6E0E
:101E7000D8B441EF0FF0200E9DEC10F00B2E3BEF8D
:101E80000FF0630E9DEC10F00950D8B44EEF0FF038
:101E9000200E9DEC10F0092E48EF0FF07C0E9DEC0B
:101EA00010F0200E9DEC10F00A2E51EF0FF0200ED6
:101EB0009DEC10F097EC24F05EEF0FF02850050E2B
:101EC000D8A4C80E6D6F27502810D8B496EF0FF025
:101ED000010E275E000E285A8AB871EF0FF080EFCE
:101EE0000FF008BC96EF0FF029502A10D8B47DEF00
:101EF0000FF0010E295E000E2A5A630E8DEF0FF0CF
:101F000008B696EF0FF02AB88AEF0FF0010E2926D7
:101F1000000E2A226F0E8DEF0FF004EC10F08A866F
:101F200004EC10F08A966D2F63EF0FF012008A9880
:101F3000F29E9F51275CA0512858D8B0A8EF0FF00F
:101F40009FC127F0A0C128F03C0E476E000E486EDE
:101F5000F28E12008A98F29E9DC127F09EC128F051
:101F60003C0E476E000E486EF28E1200CBEC0FF066
:101F7000CBEC0FF0CBEC0FF0CBEC0FF0CBEC0FF089
:101F8000CBEC0FF0CBEC0FF0CBEC0FF0CBEC0FF079
:101F9000CBEC0FF01200E9EC0FF0E9EC0FF0E9ECFC
:101FA0000FF0E9EC0FF0E9EC0FF0E9EC0FF0E9ECE1
:101FB0000FF0E9EC0FF0E9EC0FF0E9EC0FF0120094
:101FC000C70ED56E5E0ED66EF294F2A4EEEF0FF051
:101FD0001200C70ED56E940ED66EF294F2A4EEEFF8
:101FE0000FF01200C70ED56E660ED66EF294F2A4F4
:101FF000EEEF0FF01200C70ED56EF50ED66EF2940E
:10200000F2A400EF10F01200C70ED56EFD0ED66ED2
:10201000F294F2A409EF10F0120022EE00F03A510F
:102020003B19D8B41FEF10F03A29400AD8B4400E3B
:10203000400AD96E3A6FDF50AD6E20EF10F09D98D8
:10204000120025EE00F03E513F19D8B433EF10F0E6
:102050003E29000AD8B4000E000AD96E3E6FDF5048
:10206000736E34EF10F0A39812000090ABA242EF11
:1020700010F00080AB98ABB83AEF10F0AB88ABA88B
:102080003EEF10F0ABA447EF10F00080AE5000B070
:102090005EEF10F023EE00F03929FA0AD8B4FA0EF8
:1020A000FA0AD96E3819D8B45CEF10F0AE50DF6E72
:1020B000D950396F5EEF10F0AE50008212000090E0
:1020C00071A26CEF10F00080719871B864EF10F09D
:1020D000718871A868EF10F071A471EF10F00080A2
:1020E000745000B088EF10F022EE40F03D29800AD5
:1020F000D8B4C00E800AD96E3C19D8B486EF10F05F
:102100007450DF6ED9503D6F88EF10F07450008628
:102110001200166E22EE00F03B29400AD8B4400EA1
:10212000400AD96ED9503A19D8B492EF10F016502F
:10213000DF6ED9503B6F16501200176E25EE00F07F
:102140003F29000AD8B4000E000AD96ED9503E19B2
:10215000D8A4B0EF10F005A8A6EF10F0B4EF10F07F
:102160001750DF6ED9503F6F17501200BAEF10F0C2
:10217000D2EF10F0E8CF31F1D8CF32F1E0CF33F128
:102180000101A1B29AEC13F0F0B0ADEC13F0F0B293
:10219000BFEC13F09E9031C1E8FF32C1D8FF33C1CC
:1021A000E0FF1000E8CF20F1D8CF21F1EACF23F1F2
:1021B000E9CF22F1E2CF25F1E1CF24F1DACF27F107
:1021C000D9CF26F1FACF28F1FBCF29F1F5CF2DF1A8
:1021D000F8CF2CF1F7CF2BF1F6CF2AF1F3CF2EF178
:1021E000F4CF2FF1E0CF30F19EBA35EC10F0ABA276
:1021F00003EF11F00000AB98ABB8FBEF10F0AB8829
:10220000ABA8FFEF10F0A4BA5FEC10F09DA80CEFA4
:1022100011F09EB80DEC10F0A3A812EF11F0A4B8C5
:1022200021EC10F09EB238EC11F020C1E8FF21C182
:10223000D8FF23C1EAFF22C1E9FF25C1E2FF24C183
:10224000E1FF27C1DAFF26C1D9FF28C1FAFF29C162
:10225000FBFF2DC1F5FF2CC1F8FF2BC1F7FF2AC1F1
:10226000F6FF2EC1F3FF2FC1F4FF30C1E0FF1000D5
:10227000028EB12BC282362F41EF11F0640E366F01
:10228000007EAE51D8A4AE079DB84DEF11F03A5183
:102290003B19D8B44DEF11F09D88A3B856EF11F05B
:1022A0003E513F19D8B456EF11F0A38810501110C9
:1022B000D8B461EF11F0010E105E000E115AB0EFAC
:1022C00011F063EF11F0BF51C011D8B470EF11F0ED
:1022D000010EBF5F000EC05BBF51C011D8B4348D7A
:1022E000122E76EF11F0058A420E126E07B087EFBC
:1022F00011F060516111D8B48EEF11F0010E605FE2
:10230000000E615B60516111D8B48EEF11F000AE28
:102310008B9000BE8B808B928FEF11F08B90B85119
:10232000B911D8B49AEF11F0010EB85F000EB95B85
:10233000A1EF11F0A16BA26B07A2A1EF11F00A0EA1
:10234000506E49504A10D8B4ACEF11F0010E495EFE
:10235000000E4A5AB0EF11F0000E9B6FB0EF11F073
:1023600047504810D8B4B9EF11F0010E475E000E87
:10237000485A4B2ED7EF11F04C50D8A4D4EF11F09F
:102380005F51000AD8B4CEEF11F0010AD8B4CEEFF5
:1023900011F0050AD8B4CEEF11F0028C4D50D8A43C
:1023A0004D060A0ED6EF11F04C06C80E4B6E090E04
:1023B00021EC24F0C4CF6AF10D0E21EC24F06A5117
:1023C000C45CD8B0E6EF11F0C4506A5D6B6F050EC7
:1023D0006B5DD8B013EF12F0620E6A5DD8A0F7EF14
:1023E00011F0689D689D689D689D59EF12F0460E3A
:1023F0006A5DD8A002EF12F06C916C836C856C97CB
:1024000059EF12F0280E6A5DD8A00DEF12F06C8122
:102410006C936C956C8759EF12F06C916C936C9582
:102420006C9759EF12F08D0E6A5DD8A01EEF12F076
:102430006C816C83689D689D36EF12F06C0E6A5D4E
:10244000D8A029EF12F06C916C83689D689D36EFDF
:1024500012F0490E6A5DD8A034EF12F06C816C93D3
:10246000689D689D36EF12F06C916C938D0EC45C84
:10247000D8A041EF12F06C856C87689D689D59EF7C
:1024800012F06C0EC45CD8A04CEF12F06C856C9707
:10249000689D689D59EF12F0490EC45CD8A057EFB3
:1024A00012F06C956C87689D689D59EF12F06C95E1
:1024B0006C9704A65EEF12F063EF12F06CA568EF64
:1024C00012F075EF12F06CB568EF12F075EF12F0C4
:1024D0009451D8B47AEF12F0942F7AEF12F004A648
:1024E000049204B604827AEF12F0010E946F04761F
:1024F0007AEF12F004A47FEF12F084EF12F06CA7D1
:1025000089EF12F096EF12F06CB789EF12F096EFA8
:1025100012F09551D8B49BEF12F0952F9BEF12F06B
:1025200004A4049004B404809BEF12F0010E956F94
:1025300004749BEF12F004AEA0EF12F0A5EF12F0BE
:102540006CA1AAEF12F0B7EF12F06CB1AAEF12F083
:10255000B7EF12F09651D8B4BCEF12F0962FBCEF43
:1025600012F004AE049A04BE048ABCEF12F0010E0D
:10257000966F047EBCEF12F004ACC1EF12F0C6EF10
:1025800012F06CA3CBEF12F0D8EF12F06CB3CBEFDC
:1025900012F0D8EF12F09751D8B4DDEF12F0972F68
:1025A000DDEF12F004AC049804BC0488DDEF12F0F7
:1025B000010E976F047CDDEF12F005A2E2EF12F03E
:1025C000E7EF12F081A2ECEF12F0F9EF12F081B216
:1025D000ECEF12F0F9EF12F0A851D8B4FEEF12F0C0
:1025E000A82FFEEF12F005A2179705B21787FEEF8E
:1025F00012F00A0EA86F0572FEEF12F005A403EFA9
:1026000013F008EF13F081A40DEF13F01AEF13F09D
:1026100081B40DEF13F01AEF13F0AD51D8B41FEFE2
:1026200013F0AD2F1FEF13F005A4129305B412831E
:102630001FEF13F00A0EAD6F05741FEF13F0450E78
:1026400021EC24F0C4CF69F18E0E695DD8A02DEF86
:1026500013F00894089A43EF13F06D0E695DD8A04B
:1026600036EF13F00884089A43EF13F02D0E695DDE
:10267000D8A03FEF13F00894088A43EF13F00884C2
:10268000088A43EF13F008A848EF13F04DEF13F05A
:1026900008A452EF13F05FEF13F008B452EF13F0F9
:1026A0005FEF13F09251D8B464EF13F0922F64EF00
:1026B00013F008A8089608B8088664EF13F0010E16
:1026C000926F087864EF13F008AE69EF13F06EEFC5
:1026D00013F008AA73EF13F080EF13F008BA73EF4A
:1026E00013F080EF13F09351D8B485EF13F0932FCC
:1026F00085EF13F008AE089C08BE088C85EF13F038
:10270000010E936F087E85EF13F068513F0B010FA8
:102710004F6E372F95EF13F0C80E376F0188582F83
:1027200095EF13F0050E586F0686C2B295EF13F0C1
:102730009E9212004E2A4EA4ABEF13F04E6A02A4F2
:10274000A4EF13F0020E5D6F02A6A9EF13F0020EC4
:102750005E6F02840286A1921200A42B01BA028845
:10276000018AA1B29AEC13F0B2CF46F1B3CF47F190
:102770004EC048F1A1B2B1EF13F0F0901200A92BB6
:1027800001BC028A018CA1B29AEC13F0B2CF4FF1D6
:10279000B3CF50F14EC051F1A1B2C3EF13F0F0929C
:1027A0001200821CE8AAE896E8BAE8860F0B12002D
:1027B000FF0E416F426F1200421B080E436FD8900C
:1027C00041334233D8A0E9EF13F0A00E411B010EB4
:1027D000421B432FDFEF13F01200F29EF2BEEDEF2B
:1027E00013F03DC13CF1F28E009612007FEC14F024
:1027F0003250300F9DEC10F03150300F9DEC10F046
:102800003050300F9DEC10F02F50300F9DEC10F039
:102810002E50300F9DEC10F012007FEC14F0305071
:10282000300F9DEC10F02F50300F9DEC10F02E501B
:10283000300F9DEC10F01200200E9DEC10F0200ED9
:102840009DEC10F0200E9DEC10F01200200E9DEC7F
:1028500010F03A0E9DEC10F0200E9DEC10F01200DE
:102860002E502B6E2C6A2F50386E396A3A6A3B6AAA
:102870003C6A0A0E3D6E3E6A3F6A406A416A46EC17
:1028800015F038502B2639502C223050386E396ACA
:102890003A6A3B6A3C6A640E3D6E000E3E6E3F6AC9
:1028A000406A416A46EC15F038502B2639502C22EC
:1028B0003150386E396A3A6A3B6A3C6AE80E3D6EBE
:1028C000030E3E6E3F6A406A416A46EC15F038508E
:1028D0002B2639502C223250386E396A3A6A3B6ABC
:1028E0003C6A100E3D6E270E3E6E3F6A406A416A9A
:1028F00046EC15F038502B2639502C2212002E6A47
:102900002F6A306A316A326A100E2B5E270E2C5AFB
:10291000D8A08EEF14F0322A84EF14F0100E2B267C
:10292000270E2C22E80E2B5E030E2C5AD8A09CEF0B
:1029300014F0312A92EF14F0E80E2B26030E2C220D
:10294000640E2B5E000E2C5AD8A0AAEF14F0302A89
:10295000A0EF14F0640E2B26000E2C220A0E2B5E24
:10296000D8A0B6EF14F02F2AAEEF14F00A0E2B24E5
:102970002E6E12002E6A2F6A306A316A326A336A0A
:10298000346A356A800E2B5E960E2C5A980E2D5A9C
:10299000D8A0CEEF14F0352AC2EF14F0800E2B260B
:1029A000960E2C22980E2D22400E2B5E420E2C5A93
:1029B0000F0E2D5AD8A0E0EF14F0342AD4EF14F003
:1029C000400E2B26420E2C220F0E2D22A00E2B5E27
:1029D000860E2C5A010E2D5AD8A0F2EF14F0332A8D
:1029E000E6EF14F0A00E2B26860E2C22010E2D22CF
:1029F000100E2B5E270E2C5A000E2D5AD8A004EF75
:102A000015F0322AF8EF14F0100E2B26270E2C2288
:102A1000E80E2B5E030E2C5AD8A012EF15F0312AC7
:102A200008EF15F0E80E2B26030E2C22640E2B5E09
:102A3000000E2C5AD8A020EF15F0302A16EF15F012
:102A4000640E2B26000E2C220A0E2B5ED8A02CEF33
:102A500015F02F2A24EF15F00A0E2B242E6E1200EB
:102A60003D5038263E5039223F503A2240503B22BA
:102A700041503C2212003D50385E3E50395A3F5082
:102A80003A5A40503B5A41503C5A120036923696C0
:102A900038C042F039C043F03AC044F03BC045F082
:102AA0003CC046F0386A396A3A6A3B6A3C6A280E8A
:102AB000376E46324532443243324232368436A68D
:102AC0003694D8A0369436B43682D8B030EC15F0AF
:102AD000D8B03682D8903D363E363F364036413605
:102AE000D8B03686372E59EF15F0120036923D5089
:102AF0003E103F1040104110D8B4368238C042F02A
:102B000039C043F03AC044F03BC045F03CC046F009
:102B1000386A396A3A6A3B6A3C6A280E376E42362E
:102B20004336443645364636383639363A363B36FD
:102B30003C363BEC15F03688D8A03698D8A030EC5F
:102B400015F0D88036A8D890372E8FEF15F0423682
:102B5000433644364536463642C038F043C039F035
:102B600044C03AF045C03BF046C03CF012008B96A2
:102B70000000000000000000000000000000000055
:102B80000000000000000000948800000000000029
:102B90000000000000000000000000000000000035
:102BA00000008B8600000000000000000000000014
:102BB0000000000000000000000000008B989498C6
:102BC0000000000000000000000000000000000005
:102BD00000000000000000009B0E1E6E080E1F6E1D
:102BE0008B960000000000000000000000000000C4
:102BF000000000000000000000001E36D8B011EFF9
:102C000016F08B989498000000000000000000006F
:102C100000000000000000000000000000001EEFA7
:102C200016F0948800000000000000000000000082
:102C30000000000000000000000000008B86000083
:102C40000000000000000000000000000000000084
:102C50000000000000001F2EF0EF15F08B96000022
:102C60000000000000000000000000000000000064
:102C700000000000000094888B8600000000000027
:102C80000000000000000000000000000000000044
:102C9000000082B89CEF23F012008B960000000029
:102CA0000000000000000000000000000000000024
:102CB000000000009488080E1F6E8B860000000044
:102CC0000000000000000000000000000000000004
:102CD00000000000D88082A8D8901E368B96000095
:102CE00000000000000000000000000000000000E4
:102CF0000000000000001F2E5DEF16F01E508B96A6
:102D000000000000000000000000000000000000C3
:102D100000000000000000008B9894980000000064
:102D200000000000000000000000000000000000A3
:102D3000000000008B860000000000000000000082
:102D40000000000000000000000000000000120071
:102D50008B96000000000000000000000000000052
:102D6000000000000000000000009488080E1F6EA4
:102D70008B86000000000000000000000000000042
:102D800000000000000000000000D88082A8D89059
:102D90001E368B96000000000000000000000000BE
:102DA0000000000000000000000000001F2EB8EF2F
:102DB00016F01E508B96000000000000000000007E
:102DC00000000000000000000000000000009488E7
:102DD00000000000000000000000000000000000F3
:102DE00000000000000000008B86000000000000D2
:102DF00000000000000000000000000000000000D3
:102E0000000012008B96000000000000000000008F
:102E10000000000000000000000000000000948896
:102E200000000000000000000000000000000000A2
:102E300000000000000000008B8600000000000081
:102E40000000000000000000000000000000000082
:102E500000008B9894980000000000000000000023
:102E60000000000000000000000000000000850ECF
:102E70001E6E080E1F6E8B96000000000000000002
:102E80000000000000000000000000000000000042
:102E90001E36D8B05CEF17F08B98949800000000B5
:102EA0000000000000000000000000000000000022
:102EB0000000000069EF17F0948800000000000097
:102EC0000000000000000000000000000000000002
:102ED00000008B86000000000000000000000000E1
:102EE0000000000000000000000000001F2E3BEF6B
:102EF00017F08B96000000000000000000000000AA
:102F000000000000000000000000000094888B8694
:102F100000000000000000000000000000000000B1
:102F2000000000000000000082B89CEF23F01200B7
:102F30008B96000000000000000000000000000070
:102F4000000000000000000000009488080E1F6EC2
:102F50008B86000000000000000000000000000060
:102F600000000000000000000000D88082A8D89077
:102F70001E368B96000000000000000000000000DC
:102F80000000000000000000000000001F2EA8EF5D
:102F900017F01E508B96000000000000000000009B
:102FA00000000000000000000000000000008B98FE
:102FB00094980000000000000000000000000000E5
:102FC000000000000000000000008B8600000000F0
:102FD00000000000000000000000000000000000F1
:102FE0000000000012008B960000000000000000AE
:102FF00000000000000000000000000000000000D1
:103000009488080E1F6E8B860000000000000000F0
:1030100000000000000000000000000000000000B0
:10302000D88082A8D8901E368B9600000000000041
:103030000000000000000000000000000000000090
:1030400000001F2E03EF18F01E508B9600000000AA
:103050000000000000000000000000000000000070
:103060000000000094880000000000000000000044
:1030700000000000000000000000000000008B863F
:103080000000000000000000000000000000000040
:10309000000000000000000012004E0E8B960000A1
:1030A0000000000000000000000000000000000020
:1030B00000000000000094880000000000000000F4
:1030C0000000000000000000000000000000000000
:1030D0008B860000000000000000000000000000DF
:1030E000000000000000000000008B989498000091
:1030F00000000000000000000000000000000000D0
:103100000000000000001E6E080E1F6E8B9600006F
:1031100000000000000000000000000000000000AF
:103120000000000000001E36D8B0A7EF18F08B9802
:103130009498000000000000000000000000000063
:1031400000000000000000000000B4EF18F09488B8
:10315000000000000000000000000000000000006F
:1031600000000000000000008B860000000000004E
:10317000000000000000000000000000000000004F
:1031800000001F2E86EF18F08B9600000000000054
:10319000000000000000000000000000000000002F
:1031A000000094888B8600000000000000000000F2
:1031B000000000000000000000000000000082B8D5
:1031C0009CEF23F012001E6E080E1F6E8B960000FF
:1031D00000000000000000000000000000000000EF
:1031E0000000000000001E36D8B007EF19F08B98E1
:1031F00094980000000000000000000000000000A3
:103200000000000000000000000014EF19F0948896
:1032100000000000000000000000000000000000AE
:1032200000000000000000008B860000000000008D
:10323000000000000000000000000000000000008E
:1032400000001F2EE6EF18F08B9600000000000033
:10325000000000000000000000000000000000006E
:10326000000094888B860000000000000000000031
:10327000000000000000000000000000000082B814
:103280009CEF23F012000F0E18161950F00B1812B5
:1032900018501E6E080E1F6E8B9600000000000076
:1032A000000000000000000000000000000000001E
:1032B00000001E36D8B06DEF19F08B98949800007E
:1032C00000000000000000000000000000000000FE
:1032D0000000000000007AEF19F094880000000060
:1032E00000000000000000000000000000000000DE
:1032F000000000008B8600000000000000000000BD
:1033000000000000000000000000000000001F2E70
:103310004CEF19F08B960000000000000000000048
:103320000000000000000000000000000000948881
:103330008B8600000000000000000000000000007C
:103340000000000000000000000082B89CEF23F0A5
:103350001850E8841E6E080E1F6E8B960000000049
:10336000000000000000000000000000000000005D
:10337000000000001E36D8B0CEEF19F08B9894985C
:10338000000000000000000000000000000000003D
:103390000000000000000000DBEF19F0948800003E
:1033A000000000000000000000000000000000001D
:1033B0000000000000008B860000000000000000FC
:1033C00000000000000000000000000000000000FD
:1033D0001F2EADEF19F08B960000000000000000DA
:1033E00000000000000000000000000000000000DD
:1033F00094888B86000000000000000000000000A0
:1034000000000000000000000000000082B89CEFF7
:1034100023F018501E6E080E1F6E8B9600000000E1
:10342000000000000000000000000000000000009C
:10343000000000001E36D8B02EEF1AF08B9894983A
:10344000000000000000000000000000000000007C
:1034500000000000000000003BEF1AF0948800001C
:10346000000000000000000000000000000000005C
:103470000000000000008B8600000000000000003B
:10348000000000000000000000000000000000003C
:103490001F2E0DEF1AF08B960000000000000000B8
:1034A000000000000000000000000000000000001C
:1034B00094888B86000000000000000000000000DF
:1034C00000000000000000000000000082B89CEF37
:1034D00023F012000F0E18161938F00B181218509E
:1034E0001E6E080E1F6E8B9600000000000000008C
:1034F00000000000000000000000000000000000CC
:103500001E36D8B094EF1AF08B9894980000000003
:1035100000000000000000000000000000000000AB
:1035200000000000A1EF1AF09488000000000000E5
:10353000000000000000000000000000000000008B
:1035400000008B860000000000000000000000006A
:103550000000000000000000000000001F2E73EFBC
:103560001AF08B9600000000000000000000000030
:1035700000000000000000000000000094888B861E
:10358000000000000000000000000000000000003B
:10359000000000000000000082B89CEF23F01850EB
:1035A000E8841E6E080E1F6E8B960000000000005F
:1035B000000000000000000000000000000000000B
:1035C00000001E36D8B0F5EF1AF08B9894980000E2
:1035D00000000000000000000000000000000000EB
:1035E00000000000000002EF1BF0948800000000C3
:1035F00000000000000000000000000000000000CB
:10360000000000008B8600000000000000000000A9
:1036100000000000000000000000000000001F2E5D
:10362000D4EF1AF08B9600000000000000000000AC
:10363000000000000000000000000000000094886E
:103640008B86000000000000000000000000000069
:103650000000000000000000000082B89CEF23F092
:1036600018501E6E080E1F6E8B96000000000000A2
:10367000000000000000000000000000000000004A
:1036800000001E36D8B055EF1BF08B9894980000C0
:10369000000000000000000000000000000000002A
:1036A00000000000000062EF1BF0948800000000A2
:1036B000000000000000000000000000000000000A
:1036C000000000008B8600000000000000000000E9
:1036D00000000000000000000000000000001F2E9D
:1036E00034EF1BF08B96000000000000000000008B
:1036F00000000000000000000000000000009488AE
:103700008B860000000000000000000000000000A8
:103710000000000000000000000082B89CEF23F0D1
:1037200012008B9600000000000000000000000066
:10373000000000000000000000000000948800006D
:103740000000000000000000000000000000000079
:103750000000000000008B86000000000000000058
:103760000000000000000000000000000000000059
:103770008B989498000000000000000000000000FA
:103780000000000000000000000000001C341D3498
:103790001E6E1E340E0BA0091E6E080E1F6E8B9639
:1037A0000000000000000000000000000000000019
:1037B00000000000000000001E36D8B0F0EF1BF043
:1037C0008B989498000000000000000000000000AA
:1037D000000000000000000000000000FDEF1BF0F2
:1037E00094880000000000000000000000000000BD
:1037F000000000000000000000008B8600000000B8
:1038000000000000000000000000000000000000B8
:10381000000000001F2ECFEF1BF08B960000000071
:103820000000000000000000000000000000000098
:103830000000000094888B8600000000000000005B
:103840000000000000000000000000000000000078
:1038500082B89CEF23F01C507F0B1E6E080E1F6E6B
:103860008B96000000000000000000000000000037
:10387000000000000000000000001E36D8B051EF2C
:103880001CF08B98949800000000000000000000DD
:1038900000000000000000000000000000005EEFDB
:1038A0001CF09488000000000000000000000000F0
:1038B0000000000000000000000000008B860000F7
:1038C00000000000000000000000000000000000F8
:1038D0000000000000001F2E30EF1CF08B9600004F
:1038E00000000000000000000000000000000000D8
:1038F00000000000000094888B860000000000009B
:1039000000000000000000000000000000000000B7
:10391000000082B89CEF23F01B501E6E080E1F6E35
:103920008B96000000000000000000000000000076
:10393000000000000000000000001E36D8B0B1EF0B
:103940001CF08B989498000000000000000000001C
:103950000000000000000000000000000000BEEFBA
:103960001CF094880000000000000000000000002F
:103970000000000000000000000000008B86000036
:103980000000000000000000000000000000000037
:103990000000000000001F2E90EF1CF08B9600002E
:1039A0000000000000000000000000000000000017
:1039B00000000000000094888B86000000000000DA
:1039C00000000000000000000000000000000000F7
:1039D000000082B89CEF23F08B96000000000000EE
:1039E00000000000000000000000000000000000D7
:1039F00000009488000000000000000000000000AB
:103A00000000000000000000000000008B860000A5
:103A100000000000000000000000000000000000A6
:103A20000000000000008B98949800000000000047
:103A30000000000000000000000000000000000086
:103A400000001C341D341E6E1E340E0BA1091E6EA8
:103A5000080E1F6E8B9600000000000000000000A2
:103A600000000000000000000000000000001E3602
:103A7000D8B04BEF1DF08B98949800000000000028
:103A80000000000000000000000000000000000036
:103A9000000058EF1DF094880000000000000000B6
:103AA0000000000000000000000000000000000016
:103AB0008B860000000000000000000000000000F5
:103AC000000000000000000000001F2E2AEF1DF083
:103AD0008B960000000000000000000000000000C5
:103AE0000000000000000000000094888B860000A9
:103AF00000000000000000000000000000000000C6
:103B000000000000000082B89CEF23F012008B96AA
:103B100000000000000000000000000000000000A5
:103B20000000000000000000948800000000000079
:103B30000000000000000000000000000000000085
:103B400000008B8600000000000000000000000064
:103B50000000000000000000000000008B98949816
:103B60000000000000000000000000000000000055
:103B700000000000000000001C341D341E6E1E34C6
:103B80000E0BA0091E6E080E1F6E8B960000000023
:103B90000000000000000000000000000000000025
:103BA000000000001E36D8B0E6EF1DF08B98949808
:103BB0000000000000000000000000000000000005
:103BC0000000000000000000F3EF1DF094880000EA
:103BD00000000000000000000000000000000000E5
:103BE0000000000000008B860000000000000000C4
:103BF00000000000000000000000000000000000C5
:103C00001F2EC5EF1DF08B96000000000000000085
:103C100000000000000000000000000000000000A4
:103C200094888B8600000000000000000000000067
:103C300000000000000000000000000082B89CEFBF
:103C400023F01C507F0B1E6E080E1F6E8B9600001B
:103C50000000000000000000000000000000000064
:103C60000000000000001E36D8B047EF1EF08B9811
:103C70009498000000000000000000000000000018
:103C80000000000000000000000054EF1EF09488C7
:103C90000000000000000000000000000000000024
:103CA00000000000000000008B8600000000000003
:103CB0000000000000000000000000000000000004
:103CC00000001F2E26EF1EF08B9600000000000063
:103CD00000000000000000000000000000000000E4
:103CE000000094888B8600000000000000000000A7
:103CF000000000000000000000000000000082B88A
:103D00009CEF23F01B501E6E080E1F6E8B9600005A
:103D100000000000000000000000000000000000A3
:103D20000000000000001E36D8B0A7EF1EF08B98F0
:103D30009498000000000000000000000000000057
:103D400000000000000000000000B4EF1EF09488A6
:103D50000000000000000000000000000000000063
:103D600000000000000000008B8600000000000042
:103D70000000000000000000000000000000000043
:103D800000001F2E86EF1EF08B9600000000000042
:103D90000000000000000000000000000000000023
:103DA000000094888B8600000000000000000000E6
:103DB000000000000000000000000000000082B8C9
:103DC0009CEF23F012001E6E080E1F6E8B960000F3
:103DD00000000000000000000000000000000000E3
:103DE0000000000000001E36D8B007EF1FF08B98CF
:103DF0009498000000000000000000000000000097
:103E00000000000000000000000014EF1FF0948884
:103E100000000000000000000000000000000000A2
:103E200000000000000000008B8600000000000081
:103E30000000000000000000000000000000000082
:103E400000001F2EE6EF1EF08B9600000000000021
:103E50000000000000000000000000000000000062
:103E6000000094888B860000000000000000000025
:103E7000000000000000000000000000000082B808
:103E80009CEF23F012008B96000000000000000061
:103E90000000000000000000000000000000000022
:103EA0009488080E1F6E8B86000000000000000042
:103EB0000000000000000000000000000000000002
:103EC000D88082A8D8901E368B9600000000000093
:103ED00000000000000000000000000000000000E2
:103EE00000001F2E53EF1FF01E508B9600000000A5
:103EF00000000000000000000000000000000000C2
:103F0000000000008B989498000000000000000062
:103F100000000000000000000000000000000000A1
:103F20008B86000000000000000000000000000080
:103F30000000000000000000000012008B9600004E
:103F40000000000000000000000000000000000071
:103F50000000000000009488080E1F6E8B86000091
:103F60000000000000000000000000000000000051
:103F7000000000000000D88082A8D8901E368B96E2
:103F80000000000000000000000000000000000031
:103F900000000000000000001F2EAEEF1FF01E50BA
:103FA0008B960000000000000000000000000000F0
:103FB00000000000000000000000948800000000E5
:103FC00000000000000000000000000000000000F1
:103FD000000000008B8600000000000000000000D0
:103FE00000000000000000000000000000001200BF
:103FF000196E189043EC19F06AEC1AF01200188050
:10400000196E43EC19F06AEC1AF012008B9600005E
:1040100000000000000000000000000000000000A0
:104020000000000000009488000000000000000074
:104030000000000000000000000000000000000080
:104040008B8600000000000000000000000000005F
:10405000000000000000000000008B989498000011
:104060000000000000000000000000000000000050
:10407000000000000000A00E1E6E080E1F6E8B9642
:104080000000000000000000000000000000000030
:1040900000000000000000001E36D8B060EF20F0E5
:1040A0008B989498000000000000000000000000C1
:1040B0000000000000000000000000006DEF20F094
:1040C00094880000000000000000000000000000D4
:1040D000000000000000000000008B8600000000CF
:1040E00000000000000000000000000000000000D0
:1040F000000000001F2E3FEF20F08B960000000014
:1041000000000000000000000000000000000000AF
:104110000000000094888B86000000000000000072
:10412000000000000000000000000000000000008F
:1041300082B89CEF23F01B501E6E080E1F6E8B96EC
:10414000000000000000000000000000000000006F
:1041500000000000000000001E36D8B0C0EF20F0C4
:104160008B98949800000000000000000000000000
:10417000000000000000000000000000CDEF20F073
:104180009488000000000000000000000000000013
:10419000000000000000000000008B86000000000E
:1041A000000000000000000000000000000000000F
:1041B000000000001F2E9FEF20F08B9600000000F3
:1041C00000000000000000000000000000000000EF
:1041D0000000000094888B860000000000000000B2
:1041E00000000000000000000000000000000000CF
:1041F00082B89CEF23F08B960000000000000000C6
:1042000000000000000000000000000000000000AE
:104210009488000000000000000000000000000082
:10422000000000000000000000008B86000000007D
:10423000000000000000000000000000000000007E
:10424000000000008B98949800000000000000001F
:10425000000000000000000000000000000000005E
:10426000A10E1E6E080E1F6E8B960000000000004F
:10427000000000000000000000000000000000003E
:1042800000001E36D8B055EF21F08B9894980000AE
:10429000000000000000000000000000000000001E
:1042A00000000000000062EF21F094880000000090
:1042B00000000000000000000000000000000000FE
:1042C000000000008B8600000000000000000000DD
:1042D00000000000000000000000000000001F2E91
:1042E00034EF21F08B960000000000000000000079
:1042F00000000000000000000000000000009488A2
:104300008B8600000000000000000000000000009C
:104310000000000000000000000082B89CEF23F0C5
:1043200012008B960000000000000000000000005A
:104330000000000000000000000000009488000061
:10434000000000000000000000000000000000006D
:104350000000000000008B8600000000000000004C
:10436000000000000000000000000000000000004D
:104370008B989498000000000000000000000000EE
:10438000000000000000000000000000A00E1E6EF3
:10439000080E1F6E8B960000000000000000000059
:1043A00000000000000000000000000000001E36B9
:1043B000D8B0EBEF21F08B9894980000000000003B
:1043C00000000000000000000000000000000000ED
:1043D0000000F8EF21F094880000000000000000C9
:1043E00000000000000000000000000000000000CD
:1043F0008B860000000000000000000000000000AC
:10440000000000000000000000001F2ECAEF21F095
:104410008B9600000000000000000000000000007B
:104420000000000000000000000094888B8600005F
:10443000000000000000000000000000000000007C
:1044400000000000000082B89CEF23F01B501E6E9D
:10445000080E1F6E8B960000000000000000000098
:1044600000000000000000000000000000001E36F8
:10447000D8B04BEF22F08B98949800000000000019
:10448000000000000000000000000000000000002C
:10449000000058EF22F094880000000000000000A7
:1044A000000000000000000000000000000000000C
:1044B0008B860000000000000000000000000000EB
:1044C000000000000000000000001F2E2AEF22F074
:1044D0008B960000000000000000000000000000BB
:1044E0000000000000000000000094888B8600009F
:1044F00000000000000000000000000000000000BC
:1045000000000000000082B89CEF23F012001E6E35
:10451000080E1F6E8B9600000000000000000000D7
:1045200000000000000000000000000000001E3637
:10453000D8B0ABEF22F08B989498000000000000F8
:10454000000000000000000000000000000000006B
:104550000000B8EF22F09488000000000000000086
:10456000000000000000000000000000000000004B
:104570008B8600000000000000000000000000002A
:10458000000000000000000000001F2E8AEF22F053
:104590008B960000000000000000000000000000FA
:1045A0000000000000000000000094888B860000DE
:1045B00000000000000000000000000000000000FB
:1045C00000000000000082B89CEF23F012008B96E0
:1045D00000000000000000000000000000000000DB
:1045E00000000000000000009488080E1F6E8B86FB
:1045F00000000000000000000000000000000000BB
:104600000000000000000000D88082A8D8901E366C
:104610008B96000000000000000000000000000079
:10462000000000000000000000001F2EF7EF22F045
:104630001E508B96000000000000000000000000EB
:104640000000000000000000000000008B9894981B
:10465000000000000000000000000000000000005A
:1046600000000000000000008B8600000000000039
:10467000000000000000000000000000000000003A
:10468000000012008B9600000000000000000000F7
:1046900000000000000000000000000000009488FE
:1046A000080E1F6E8B860000000000000000000056
:1046B0000000000000000000000000000000D880A2
:1046C00082A8D8901E368B960000000000000000E3
:1046D00000000000000000000000000000000000DA
:1046E0001F2E52EF23F01E508B960000000000009A
:1046F00000000000000000000000000000000000BA
:10470000000094880000000000000000000000008D
:104710000000000000000000000000008B86000088
:104720000000000000000000000000000000000089
:10473000000000000000120005808B9600000000C1
:104740000000000000000000000000000000000069
:10475000000000008B98949800000000000000000A
:104760000000000000000000000000000000000049
:104770008B86000000000000000000000000000028
:10478000000000000000000000009488000000000D
:104790000000000000000000000000000000000019
:1047A000000000001200000000008B9600000000D6
:1047B00000000000000000000000000000000000F9
:1047C000000000008B98949800000000000000009A
:1047D00000000000000000000000000000000000D9
:1047E0008B860000000000000000000000000000B8
:1047F000000000000000000000009488000000009D
:1048000000000000000000000000000000000000A8
:10481000000000001200096E093816EC24F009505F
:1048200016EC24F0200E9DEC10F012000F0B0A6E17
:104830000A0E0A5C300ED8B0370E0A249DEC10F038
:104840001200C26EC282C2B223EF24F012000588A9
:104850002DEF24F005982DEF24F00900F550D8B481
:1048600036EF24F09DEC10F02DEF24F005881200B7
:10487000800EF8EC1FF0F2EC0FF00900F550D8B400
:1048800046EF24F0FFEC1FF03DEF24F01200C00EC5
:10489000F8EC1FF0F2EC0FF00900F550D8B455EF2A
:1048A00024F0FFEC1FF04CEF24F01200B751F8ECAD
:1048B0001FF0F2EC0FF07FEC14F03250300FFFECF1
:1048C0001FF03150300FFFEC1FF03050300FFFEC75
:1048D0001FF02F50300FFFEC1FF02E50300FFFEC69
:1048E0001FF01200B751F8EC1FF0F2EC0FF07FEC64
:1048F00014F03150300FFFEC1FF03050300FFFEC50
:104900001FF02F50300FFFEC1FF02E50300FFFEC38
:104910001FF012004F0E9DEC10F0410E9DEC10F0B8
:10492000310E9DEC10F0370E9DEC10F012000D0EC4
:104930009DEC10F00A0E9DEC10F0120001AACEEFD3
:1049400024F0F29E019A46C149F147C14AF148C19B
:104950004BF1029402804C51495DA56F4D514A596B
:10496000A66F4E514B59A76F49C14CF14AC14DF149
:104970004BC14EF15D51D8B4C4EF24F05D07FF0E7A
:10498000A46BA56FA66FA76F030EA7B5A717F28E2E
:10499000D4EC0AF0C80EB86F000EB96F120001AC6B
:1049A000F8EF24F0F29E019C4FC152F150C153F137
:1049B00051C154F1029602825551525DAA6F56516F
:1049C0005359AB6F57515459030BAC6F52C155F14A
:1049D00053C156F154C157F15E51D8B4F8EF24F0E9
:1049E0005E07FF0EA96BAA6FAB6FAC6FF8EF24F0F8
:1049F000F28E120002AC7DEF26F0029C5F51000A9D
:104A0000D8B411EF25F0010AD8B468EF25F0030AF5
:104A1000D8B41AEF26F0010AD8B41CEF26F041EF03
:104A200026F04D50D8A41FEF25F0280E4D6EA68E0F
:104A3000F86A080EF76ED00EF66E27EC24F0B1C1BE
:104A40002BF02C6A0DEC14F026EC14F0A1C12BF025
:104A5000A2C12CF0F6EC13F026EC14F0F29E99C1F2
:104A60002BF09AC12CF0F28EF6EC13F026EC14F039
:104A7000F29E90C1E9FF91C1EAFFEECFE8FFEECFD1
:104A80002BF0EECF2CF0F28EF6EC13F026EC14F0B7
:104A9000F6EC13F0058826EC14F0450E9DEC10F0B2
:104AA0003D0E9DEC10F0300E310E9DEC10F026EC1A
:104AB00014F0520E9DEC10F03D0E9DEC10F07F0BAB
:104AC000300F9DEC10F0059897EC24F07DEF26F068
:104AD000B1C12BF02C6A0DEC14F026EC14F0B2C12D
:104AE0002BF02C6A0DEC14F026EC14F001EE00F023
:104AF000EECFE8FF0BEC24F0EECFE8FF0BEC24F058
:104B0000EECFE8FF0BEC24F0280E9DEC10F0300EF9
:104B100002B5310E9DEC10F0300E02B3310E9DEC5B
:104B200010F0300E02B1310E9DEC10F0290E9DEC0C
:104B300010F0200E9DEC10F0EECFE8FF0BEC24F00F
:104B4000EECFE8FF0BEC24F0EECFE8FF0BEC24F007
:104B5000EECFE8FF0BEC24F0EECFE8FF0BEC24F0F7
:104B6000EECFE8FF0BEC24F0EECFE8FF0BEC24F0E7
:104B7000EECFE8FF0BEC24F0EECFE8FF0BEC24F0D7
:104B8000EECFE8FF0BEC24F0EECFE8FF0BEC24F0C7
:104B9000EECFE8FF0BEC24F0EECFE8FF0BEC24F0B7
:104BA0003A0E9DEC10F0200E9DEC10F0EECFE8FFD9
:104BB0000BEC24F0EECFE8FF0BEC24F0EECFE8FF97
:104BC0000BEC24F0EECFE8FF0BEC24F0EECFE8FF87
:104BD0000BEC24F0EECFE8FF0BEC24F0EECFE8FF77
:104BE0000BEC24F0EECFE8FF0BEC24F0EECFE8FF67
:104BF0000BEC24F0EECFE8FF0BEC24F0EECFE8FF57
:104C00000BEC24F0EECFE8FF0BEC24F0EECFE8FF46
:104C10000BEC24F0EECFE8FF0BEC24F0EECFE8FF36
:104C20000BEC24F0EECFE8FF0BEC24F097EC24F033
:104C30007DEF26F07DEF26F04D50D8A42CEF26F026
:104C4000280E4D6EA68EF86A080EF76EBC0EF66E34
:104C500027EC24F03FEF26F0B1C12BF02C6A0DECCD
:104C600014F026EC14F02C6A0DEC14F026EC14F081
:104C70009CC12BF02C6A0DEC14F097EC24F07DEF26
:104C800026F04D50D8A451EF26F0280E4D6EA68E7A
:104C9000F86A080EF76EF80EF66E27EC24F07DEF3A
:104CA00026F002A07DEF26F00290AAC12BF0ABC146
:104CB00000F0BAEC14F03550300F9DEC10F0345089
:104CC000300F9DEC10F03350300F9DEC10F032504F
:104CD000300F9DEC10F03150300F9DEC10F0305043
:104CE000300F9DEC10F02F50300F9DEC10F02E5037
:104CF000300F9DEC10F097EC24F012002B50995DD2
:104D0000386E2C509A59396ED8A093EF26F089EF5F
:104D100026F08A98E00E38143910010ED8A4050E3A
:104D2000276EA3EF26F08A88381E391E010E38261A
:104D3000000E3922E00E38143910010ED8A4050EE9
:104D4000276EA3EF26F01200F29EF2BEA4EF26F02B
:104D500039C138F1F28E120038513919D8A4D880EF
:104D6000D8B4D890D8B4C7EF26F0BCEF26F03851AD
:104D70003919D8B4B7EF26F023EE00F03829FA0A33
:104D8000D8B4FA0EFA0AD96E386FDF50D880120004
:104D90003C513D19D8A4D880D8B4D890D8B4E3EF0A
:104DA00026F0D8EF26F03C513D19D8B4D3EF26F0C9
:104DB00022EE40F03C29800AD8B4C00E800AD96E99
:104DC0003C6FDF50D88012003491FA0E556E000E01
:104DD000546E1200ACEC26F0D8A032EF27F0566EDD
:104DE0005550D8B407EF27F024EE00F05450D96E98
:104DF000542A5650DF6E55060D0AD8B407EF27F037
:104E0000070AD8B407EF27F0EAEF26F0348324EE40
:104E100000F0FA0E576E5550575E572E14EF27F0DC
:104E2000E4EC26F0EAEF26F0DF50349533EC27F07F
:104E300034A51FEF27F0E4EC26F0EAEF26F04BEC68
:104E400027F0A68EF86A060EF76E2E0EF66E140E7A
:104E50005C6E88EC27F0D8B030EF27F0FF0E5A6E6A
:104E60005A503481120034B546EF27F0DF50200A43
:104E7000D8B441EF27F0290AD8B441EF27F046EF24
:104E800027F0D92A572E33EF27F03485D950586EA2
:104E9000596ADF50120034B559EF27F0D7EC27F0EC
:104EA000D8A059EF27F0D92A592A572E4BEF27F0CF
:104EB0003485DF505952120034B56AEF27F02EECDA
:104EC00028F0D8A06AEF27F0D92A592A572E5CEF8C
:104ED00027F03485DF505952120034B57BEF27F0AC
:104EE00054EC28F0D8A07BEF27F0D92A592A572E66
:104EF0006DEF27F03485DF505952120034B586EF3C
:104F000027F0D92A572E86EF27F03485DF5012007C
:104F10005950D8B4B6EF27F05A6A5850D96E595044
:104F20005B6E0900F550FF0BD8B4ABEF27F0DF5CE8
:104F3000D8A4A5EF27F0D92A5B2E91EF27F009001E
:104F4000F550FF0BD8B4B9EF27F00900F550FF0B6F
:104F5000D8A4A5EF27F00900F550FF0BD8B4ABEFAC
:104F600027F00A005A2A5C2E8DEF27F0D890BAEF6E
:104F700027F0D8801200410EDF5CD8A0D4EF27F0D4
:104F80005B0EDF5CD8A0D1EF27F0610EDF5CD8A00C
:104F9000D4EF27F07B0EDF5CD8B0D4EF27F0200EE3
:104FA000DF5ED880D5EF27F0D890DF501200200EBA
:104FB000DF5C34ABD894D8B428EF28F0210EDF5C46
:104FC000D8B428EF28F0220E34A9230EDF5CD8A035
:104FD0002BEF28F02C0EDF5CD8A028EF28F02C0E49
:104FE00034AB2D0EDF5CD8A02BEF28F0300EDF5C49
:104FF000D8A028EF28F0300EDF5CD8A02BEF28F0E7
:105000003A0EDF5CD8A028EF28F03A0EDF5CD8A07B
:105010002BEF28F0410EDF5CD8A028EF28F0410EDE
:10502000DF5CD8A02BEF28F05B0EDF5CD8A028EF68
:1050300028F0610EDF5CD8A02BEF28F07B0EDF5C40
:10504000D8B02BEF28F034A728EF28F0200EDF5E31
:10505000D8802CEF28F0D890DF501200300EDF5CA3
:10506000D8A051EF28F03A0EDF5CD8A04EEF28F020
:10507000410EDF5CD8A051EF28F05B0EDF5CD8A0BA
:105080004EEF28F0610EDF5CD8A051EF28F07B0EC8
:10509000DF5CD8B051EF28F0200EDF5ED88052EFF1
:1050A00028F0D890DF501200300EDF5CD8A061EFFE
:1050B00028F03A0EDF5CD8B061EF28F0D88062EFBC
:1050C00028F0D890DF501200BB6FBB3970EC28F08D
:1050D00089EC10F0BB5170EC28F089EC10F0120054
:1050E0000F0B300FBA6F3A0EBA5D070ED8A0000E44
:1050F000BA251200FB6ABCC1BDF1BE6BD890BD37AA
:10510000BE37BD37BE37140EBD27510EBE21FA6E15
:10511000BD51F96EF6EF28F0FEEF28F007EF29F009
:105120001AEF29F025EF29F02DEF29F034EF29F0BF
:105130004BEF29F061EF29F07EEF29F08DEF29F098
:10514000A6EF29F0B9EF29F0D4EF29F0DBEF29F031
:10515000F4EF29F007EF2AF016EF2AF01DEF2AF0FE
:1051600036EF2AF049EF2AF058EF2AF05FEF2AF0E5
:1051700078EF2AF08BEF2AF091EF2BF098EF2BF0DD
:10518000AFEF2BF0C2EF2BF0D2EF2BF0DDEF2BF0D7
:10519000F4EF2BF007EF2CF029EF2CF030EF2CF090
:1051A00047EF2CF05AEF2CF0B7EF2CF0CCEF2CF0AF
:1051B0000BEF2DF012EF2DF03EEF2DF05CEF2DF008
:1051C000CEEF2DF0E1EF2DF0FBEF2DF002EF2EF002
:1051D00032EF2EF045EF2EF056EF2EF069EF2EF065
:1051E00074EF2EF086EF2EF08BEF2EF0050E586F39
:1051F000010EE8CFBCF106967AEF28F006A605EF7F
:1052000029F00696050EE8CFBCF19FEF2EF080B294
:1052100012EF29F08980A0EC2EF0030EE8CFBCF14C
:105220009FEF2EF08990C4EC2EF0040EE8CFBCF175
:105230009FEF2EF034AD23EF29F08990C4EC2EF0CF
:10524000040EE8CFBCF19FEF2EF034AD2BEF29F028
:10525000050EE8CFBCF19FEF2EF0B2EC2EF0060E5B
:10526000E8CFBCF19FEF2EF034AD49EF29F0A4EC6C
:1052700026F0349FA68EF86A040EF76E000EF66EC6
:1052800006EC2FF0B8EC2EF0E4EC26F0070EE8CF99
:10529000BCF19FEF2EF0348BEAEC26F034A156EFF0
:1052A00029F0080EE8CFBCF17AEF28F034AD5FEFBB
:1052B00029F03591310E89A0020EE8CFBCF19FEFA5
:1052C0002EF05A50010AD8A46EEF29F03583E4EC91
:1052D00026F0070EE8CFBCF17AEF28F0010AD8A437
:1052E00078EF29F03581090EE8CFBCF17CEF29F089
:1052F0003591310EE8CFBCF19FEF2EF035B386EF3C
:1053000029F00D0EE8CFBCF18BEF29F0B2EC2EF0B6
:105310000A0EE8CFBCF19FEF2EF034ADA4EF29F0D8
:10532000A4EC26F0349FA68EF86A040EF76E040EE5
:10533000F66E06EC2FF0B8EC2EF0E4EC26F00B0E37
:10534000E8CFBCF17AEF28F09FEF2EF0348BEAEC37
:1053500026F034A1B1EF29F00C0EE8CFBCF17AEFC2
:1053600028F034ADB7EF29F0310EE8CFBCF19FEF54
:105370002EF05A50020AD8A4C5EF29F0E4EC26F02A
:105380000B0EE8CFBCF17AEF28F0020AD8A4CFEFD9
:1053900029F035930D0EE8CFBCF1D2EF29F0310E94
:1053A000E8CFBCF19FEF2EF0B2EC2EF00E0EE8CF5E
:1053B000BCF19FEF2EF034ADF2EF29F0A4EC26F013
:1053C000349FA68EF86A040EF76E0A0EF66E06EC8F
:1053D0002FF0B8EC2EF0E4EC26F00F0EE8CFBCF185
:1053E0007AEF28F09FEF2EF0348BEAEC26F034A110
:1053F000FFEF29F0100EE8CFBCF17AEF28F034ADC2
:1054000005EF2AF0310EE8CFBCF19FEF2EF05A5095
:10541000000AD8A411EF2AF0110EE8CFBCF17AEF00
:1054200028F0110EE8CFBCF19FEF2EF0B2EC2EF079
:10543000120EE8CFBCF19FEF2EF034AD34EF2AF01E
:10544000A4EC26F0349FA68EF86A040EF76E160EB2
:10545000F66E06EC2FF0B8EC2EF0E4EC26F0130E0E
:10546000E8CFBCF17AEF28F09FEF2EF0348BEAEC16
:1054700026F034A141EF2AF0140EE8CFBCF17AEF08
:1054800028F034AD47EF2AF0310EE8CFBCF19FEFA2
:105490002EF05A50000AD8A453EF2AF0150EE8CF88
:1054A000BCF17AEF28F0150EE8CFBCF19FEF2EF09B
:1054B000B2EC2EF0160EE8CFBCF19FEF2EF034AD1B
:1054C00076EF2AF0A4EC26F0349FA68EF86A040E3C
:1054D000F76E1C0EF66E06EC2FF0B8EC2EF0E4EC36
:1054E00026F0170EE8CFBCF17AEF28F09FEF2EF0F0
:1054F000349BEAEC26F034A183EF2AF0180EE8CFB3
:10550000BCF17AEF28F034AD89EF2AF0310EE8CF04
:10551000BCF19FEF2EF05A50000AD8A495EF2AF064
:10552000190EE8CFBCF17AEF28F05A50120AD8A42D
:105530008CEF2BF0190EE8CFBCF133EC27F0220EE4
:10554000DF5CD8A483EF2BF07EEC27F054EC28F03E
:10555000D8A083EF2BF0300EDF5CE838CF6F7EEC05
:1055600027F054EC28F0D8A083EF2BF0300EDF5C4E
:10557000CF137EEC27F02F0EDF5CD8A483EF2BF047
:105580007EEC27F054EC28F0D8A083EF2BF0300EFF
:10559000DF5CE838CE6F7EEC27F054EC28F0D8A022
:1055A00083EF2BF0300EDF5CCE137EEC27F02F0E56
:1055B000DF5CD8A483EF2BF07EEC27F054EC28F0CE
:1055C000D8A083EF2BF0300EDF5CE838CD6F7EEC97
:1055D00027F054EC28F0D8A083EF2BF0300EDF5CDE
:1055E000CD137EEC27F02C0EDF5CD8A483EF2BF0DC
:1055F0007EEC27F054EC28F0D8A083EF2BF0300E8F
:10560000DF5CE838CC6F7EEC27F054EC28F0D8A0B3
:1056100083EF2BF0300EDF5CCC137EEC27F03A0EDC
:10562000DF5CD8A483EF2BF07EEC27F054EC28F05D
:10563000D8A083EF2BF0300EDF5CE838CB6F7EEC28
:1056400027F054EC28F0D8A083EF2BF0300EDF5C6D
:10565000CB137EEC27F03A0EDF5CD8A483EF2BF05F
:105660007EEC27F054EC28F0D8A083EF2BF0300E1E
:10567000DF5CE838CA6F7EEC27F054EC28F0D8A045
:1056800083EF2BF0300EDF5CCA137EEC27F0D06F77
:105690007EEC27F054EC28F0D8A083EF2BF0300EEE
:1056A000DF5CD16F7EEC27F054EC28F0D8A083EFBC
:1056B0002BF0300EDF5CD26FCF51C819D8A483EF26
:1056C0002BF0CE51C719D8A483EF2BF0CD51C619BA
:1056D000D8A483EF2BF0CC51C419D8A483EF2BF0BE
:1056E000CB51C35DD8B077EF2BF0C351CB5D000A2F
:1056F000D8B483EF2BF0010AD8B483EF2BF0030A60
:10570000D8B483EF2BF0FBEC0FF0E4EC26F0170E8F
:10571000E8CFBCF17AEF28F01D0EE8CFBCF19FEF87
:105720002EF0B2EC2EF01A0EE8CFBCF19FEF2EF067
:1057300034ADADEF2BF0A4EC26F0349FA68EF86AC2
:10574000040EF76E260EF66E06EC2FF0B8EC2EF077
:10575000E4EC26F01B0EE8CFBCF19FEF2EF0348B6B
:10576000EAEC26F034A1BAEF2BF01C0EE8CFBCF126
:105770007AEF28F034ADC0EF2BF0310EE8CFBCF15A
:105780009FEF2EF05A50000AD8A4CDEF2BF0C16B3A
:10579000210EE8CFBCF1D0EF2BF0310EE8CFBCF1F9
:1057A0009FEF2EF0E5EC2EF0C151D8A4DAEC2EF0EC
:1057B0001E0EE8CFBCF19FEF2EF034ADF2EF2BF0D0
:1057C000A4EC26F0349FA68EF86A040EF76E320E13
:1057D000F66E06EC2FF0B8EC2EF0E4EC26F01F0E7F
:1057E000E8CFBCF19FEF2EF0348BEAEC26F034A129
:1057F000FFEF2BF0200EE8CFBCF17AEF28F034ADAC
:1058000005EF2CF0310EE8CFBCF19FEF2EF05A508F
:10581000040AD8A411EF2CF0210EE8CFBCF127EF39
:105820002CF05A50050AD8A41BEF2CF0270EE8CF15
:10583000BCF127EF2CF01D0EE8CFBCF1C12BC151FC
:105840000D0AD8A427EF2CF0310EE8CFBCF19FEF62
:105850002EF0B8EC2EF0220EE8CFBCF19FEF2EF028
:1058600034AD45EF2CF0A4EC26F0349FA68EF86AF8
:10587000040EF76E6C0EF66E06EC2FF0BEEC2EF0FA
:10588000E4EC26F0230EE8CFBCF19FEF2EF0349B22
:10589000EAEC26F034A152EF2CF0240EE8CFBCF154
:1058A0007AEF28F034AD58EF2CF0310EE8CFBCF190
:1058B0009FEF2EF05A50000AD8A464EF2CF0000E8F
:1058C000E8CFBCF1B5EF2CF05A500B0AD8B46FEF0B
:1058D0002CF00694310EE8CFBCF1B5EF2CF033EC90
:1058E00027F06DEC27F0D9CFE9FFDACFEAFFD66BCE
:1058F000DD50010ED76FDD50D00FD703F350D62700
:105900000A0ED703F3CFD7F1592E7BEF2CF0E9CF56
:10591000D9FFEACFDAFFD86B34B5B0EF2CF07EECCC
:1059200027F02C0AD8A48CEF2CF034B5B0EF2CF073
:105930007EEC27F0220AD8A4B0EF2CF001EED9F0CB
:1059400034B5AFEF2CF07EEC27F0220AD8B4B0EFDC
:105950002CF0220AEE6ED82BD8A9A0EF2CF0D86B31
:10596000E4EC26F0250EE8CFBCF19FEF2EF0348B4F
:105970003497EAEC26F0348734A1C4EF2CF0260EDD
:10598000E8CFBCF17AEF28F034ADCAEF2CF0000E6E
:10599000E8CFBCF19FEF2EF0069224EE00F0D9067E
:1059A000F90E576E5550575E349534B501EF2DF012
:1059B0007EEC27F0EA19D8A401EF2DF034B501EF01
:1059C0002DF07EEC27F0EB19D8A401EF2DF034B5C3
:1059D00001EF2DF07EEC27F0EC19D8A401EF2DF0AB
:1059E00034B501EF2DF07EEC27F0ED19D8A401EFCE
:1059F0002DF0068234B501EF2DF07EEC27F001EF9B
:105A00002DF0270E06A22D0ED853D8B42D0EE8CFB8
:105A1000BCF19FEF2EF0B2EC2EF0280EE8CFBCF1D7
:105A20009FEF2EF0ACEC26F0D8A019EF2DF0B2ECE1
:105A30002EF034AD3CEF2DF0A4EC26F0348FA68E82
:105A4000F86A040EF76E3C0EF66E06EC2FF001EECF
:105A5000D9F0D8C1D3F1EE5089EC10F0D32F2BEF51
:105A60002DF0220E89EC10F00D0E89EC10F0B8EC40
:105A70002EF0290EE8CFBCF19FEF2EF0ACEC26F013
:105A8000D8A054EF2DF00D0AD8B43EEF2DF0070A40
:105A9000D8B43EEF2DF0340AD8A457EF2DF02A0EDB
:105AA000E8CFBCF15AEF2DF034AD5AEF2DF0310EA6
:105AB000E8CFBCF19FEF2EF0ACEC26F0D8A0C6EFFB
:105AC0002DF0200AD8A4C9EF2DF0348FA68EF86AE5
:105AD000040EF76E580EF66E06EC2FF0F5C12BF0A3
:105AE000F6C12CF07FEC14F03250300F89EC10F03E
:105AF0003150300F89EC10F03050300F89EC10F03D
:105B00002F50300F89EC10F02E50300F89EC10F030
:105B1000200E89EC10F06F0E89EC10F0660E89EC07
:105B200010F0200E89EC10F099C12BF09AC12CF0E6
:105B30007FEC14F03250300F89EC10F03150300F00
:105B400089EC10F03050300F89EC10F02F50300FEE
:105B500089EC10F02E50300F89EC10F0200E89ECFB
:105B600010F04C0E89EC10F02F0E89EC10F0480E5E
:105B700089EC10F01A0E89EC10F017EC2FF0E4EC21
:105B800026F02B0EE8CFBCF1CCEF2DF034ADCCEFEE
:105B90002DF0310EE8CFBCF19FEF2EF0349BEAECF4
:105BA00026F034A1D9EF2DF02C0EE8CFBCF17AEF1E
:105BB00028F034ADDFEF2DF0310EE8CFBCF19FEFD0
:105BC0002EF05A500A0AD8A4EDEF2DF0E4EC26F09E
:105BD0002B0EE8CFBCF1F9EF2DF00A0AD8A4F6EFAE
:105BE0002DF02D0EE8CFBCF1F9EF2DF02D0EE8CF02
:105BF000BCF19FEF2EF0BEEC2EF02E0EE8CFBCF1E4
:105C00009FEF2EF034AD30EF2EF0D76B0A0ED65F3B
:105C1000D8A00EEF2EF0D72B07EF2EF0D627A4EC4E
:105C200026F0348FA68EF86A040EF76E860EF66E96
:105C300006EC2FF0349FD751D8B422EF2EF0300F5E
:105C400089EC10F0D651300F89EC10F00D0E89EC74
:105C500010F0B8EC2EF0E4EC26F02F0EE8CFBCF1FB
:105C60009FEF2EF0349BEAEC26F034A13DEF2EF0AE
:105C7000300EE8CFBCF17AEF28F034AD43EF2EF0D0
:105C8000310EE8CFBCF19FEF2EF05A50000AD8A495
:105C90004FEF2EF0000EE8CFBCF154EF2EF0310E96
:105CA000E8CFBCF154EF2EF09FEF2EF080A261EF11
:105CB0002EF08980A6EC2EF0320EE8CFBCF19FEFDB
:105CC0002EF08990B8EC2EF0350EE8CFBCF19FEFA6
:105CD0002EF034AD23EF29F08990ACEC2EF0330E8A
:105CE000E8CFBCF19FEF2EF034AD7CEF2EF0310EFB
:105CF000E8CFBCF184EF2EF080B284EF2EF0350EA9
:105D000006A0340EE8CFBCF19FEF2EF0000EE8CFD6
:105D1000BCF19FEF2EF034AD9DEF2EF0E851D8B4DA
:105D200098EF2EF0E807020EE8CFBCF19DEF2EF0C1
:105D3000000EE8CFBCF19DEF2EF09FEF2EF0120089
:105D4000C80EBF6F000EC06F349D1200A40EBF6F4F
:105D5000010EC06F349D1200280EBF6F000EC06F81
:105D6000349D1200140EBF6F000EC06F349D1200E0
:105D7000E80EBF6F030EC06F349D1200D00EBF6FD0
:105D8000070EC06F349D1200F29EF2BEC4EF2EF0DB
:105D9000A00EBF6F0F0EC06F349DF28E1200F29EE8
:105DA000F2BECFEF2EF0500EBF6F460EC06F349D87
:105DB000F28E1200F29EF2BEDAEF2EF0E80EBF6F06
:105DC000030EC06F349DF28E1200F29EF2BEE5EF1C
:105DD0002EF0E00EBF6F2E0EC06F349DF28E1200BB
:105DE000F29EF2BEF0EF2EF0980EBF6F3A0EC06F2B
:105DF000349DF28E1200F29EF2BEFBEF2EF0680E82
:105E0000BF6F420EC06F349DF28E12000900F55034
:105E1000FF0BD8B410EF2FF089EC10F006EF2FF045
:105E200034BF16EF2FF00D0E89EC10F01200A00E0B
:105E3000BF6F8C0EC06F349D120006EE00F0E9506B
:105E4000C00F0EEC00F0EE6EE9AC1FEF2FF0120069
:105E5000FFFFFFFFFFFFFFFFFFFFFFFFFFFFFFFF52
:105E6000FFFFFFFFFFFFFFFFFFFFFFFFFFFFFFFF42
:105E7000FFFFFFFFFFFFFFFFFFFFFFFFFFFFFFFF32
:105E8000FFFFFFFFFFFFFFFFFFFFFFFFFFFFFFFF22
:0200000400F00A
:10000000E8030031323334000000AA00000400008D
:1000100004000000FF00FFFF00000000047DFFFF60
:10002000FFFFFFFFFFFFFFFFFFFFFFFFFFFFFFFFE0
:10003000FFFFFFFFFFFFFFFFFFFFFFFFFFFFFFFFD0
:100040005A62FFFFFFFFFFFFFFFFFFFFFFFFFFFF02
:10005000FFFFFFFFFFFFFFFFFFFFFFFFFFFFFFFFB0
:10006000FFFFFFFFFFFFFFFFFFFFFFFFFFFFFFFFA0
:10007000FFFFFFFFFFFFFFFFFFFFFFFFFFFFFFFF90
:100080004150502053435241544348504144FFFF94
:10009000FFFFFFFFFFFFFFFFFFFFFFFFFFFFFFFF70
:1000A000FFFFFFFFFFFFFFFFFFFFFFFFFFFFFFFF60
:1000B000FFFFFFFFFFFFFFFFFFFFFFFFFFFFFFFF50
:1000C0008C87827D787573716D696766656463621C
:1000D00061605F5E5E5D5D5C5C5B5B5A5A5959595D
:1000E00058585857575756565655555555545454B1
:1000F00054535353535352525252515151515151DF
:020000040030CA
:0E0000000023003C0099800000000FE00F403C
:020000040020DA
:08000000FFFFFFFFFFFFFFFF00
:00000001FF
